:020000040800F2
:10000000700D002065010008B3120008A50C00085F
:1000100000000000000000000000000000000000E0
:10002000000000000000000000000000E5180008CB
:100030000000000000000000B9140008051B0008C3
:1000400077010008770100087701000877010008B0
:100050007701000869070008770100088D0700088C
:10006000770100087701000877010008E50500081E
:100070007701000877010008770100087701000880
:1000800077010008770100080000000077010008F0
:100090007701000877010008770100087701000860
:1000A000770100087701000877010008A91B000804
:1000B0007701000800000000770100080000000040
:1000C00000F002F800F03EF80CA030C80838241800
:1000D0002D18A246671EAB4654465D46AC4201D180
:1000E00000F030F87E460F3E0FCCB6460126334274
:1000F00000D0FB1AA246AB4633431847AC29000098
:10010000CC290000103A02D378C878C1FAD8520737
:1001100001D330C830C101D504680C6070470000BD
:100120000023002400250026103A01D378C1FBD813
:10013000520700D330C100D50B6070471FB51FBDFB
:1001400010B510BD00F01CF91146FFF7F7FF02F0E3
:1001500005F800F034F903B4FFF7F2FF03BC00F038
:100160003BF900000748804707480047FEE7FEE7E5
:10017000FEE7FEE7FEE7FEE704480549054A064BB1
:10018000704700002D1B0008C10000087007002008
:10019000700D0020700900207009002030B5441C4B
:1001A00003E00178401C00290DD08107F9D10B4BE9
:1001B000DD0104C8D11A91432940FAD0001B0A0678
:1001C00003D0C01E30BD001B30BD0A0401D0801E0C
:1001D00030BD0902FCD0401E30BD0000010101010C
:1001E00001E004C0091F0429FBD28B0701D502805E
:1001F000801CC90700D00270704700290BD0C307CC
:1002000002D00270401C491E022904D3830702D584
:100210000280801C891EE3E70022EEE70022DFE770
:10022000002203098B422CD3030A8B4211D30023F3
:100230009C464EE003460B433CD4002243088B42CD
:1002400031D303098B421CD3030A8B4201D394465A
:100250003FE0C3098B4201D3CB01C01A524183094D
:100260008B4201D38B01C01A524143098B4201D307
:100270004B01C01A524103098B4201D30B01C01A32
:100280005241C3088B4201D3CB00C01A52418308AC
:100290008B4201D38B00C01A524143088B4201D3D9
:1002A0004B00C01A5241411A00D201465241104639
:1002B00070475DE0CA0F00D04942031000D34042AE
:1002C000534000229C4603098B422DD3030A8B42E4
:1002D00012D3FC22890112BA030A8B420CD3890182
:1002E00092118B4208D3890192118B4204D3890168
:1002F0003AD0921100E08909C3098B4201D3CB01A6
:10030000C01A524183098B4201D38B01C01A52415A
:1003100043098B4201D34B01C01A524103098B425E
:1003200001D30B01C01A5241C3088B4201D3CB0049
:10033000C01A524183088B4201D38B00C01A52412C
:10034000D9D243088B4201D34B00C01A5241411A03
:1003500000D20146634652415B10104601D3404231
:10036000002B00D54942704763465B1000D34042E2
:1003700001B50020C046C04602BD704770477047B7
:10038000754600F025F8AE46050069465346C0089C
:10039000C000854618B020B5FFF7EEFE60BC002710
:1003A0004908B6460026C0C5C0C5C0C5C0C5C0C541
:1003B000C0C5C0C5C0C5403D49008D46704710B599
:1003C0000446C046C0462046FFF7C5FE10BD0000EB
:1003D000004870470C07002001491820ABBEFEE71B
:1003E000260002007047000038B50021009100246B
:1003F0006A460F4801F0F0FC68460078002815D1E5
:1004000001F0F4FE002811D000BF0CE0204601F0FE
:10041000F9FE002805D0E100064A8918486880479F
:1004200003E0601CC4B2102CF0DB00BF38BD00003C
:100430007006002098290008054800880549884270
:1004400004D003480088401C014908807047000020
:1004500064000020FFFF000010B5002000F070FFD6
:1004600004462078052805DA608822789200104B2F
:10047000995888470F480078401C0E490870084674
:100480000078322802DD6420087006E00948007810
:100490000A2802DD642007490870074800887D218A
:1004A0000901884202DB00200349088010BD0000DA
:1004B000182A00087A0000206400002010B50024EB
:1004C000542200210C4800F0E9FE0C480078000698
:1004D0000A49497809040843084989780902084308
:1004E0000649097908430446204600F0DDFB02492D
:1004F0004031888110BD0000B8060020003300089C
:1005000010B53448C079012822D133480078401C06
:100510003149087008460078052804DA10212F4870
:1005200000F056FA21E02C480078092807DB00206B
:10053000294908701021294800F048FA15E026489A
:100540000078052811DD1021244800F03FFA0CE066
:100550002048C079022804D11021204800F038FA40
:1005600003E010211D4800F031FA1A48007A0128F2
:1005700022D11B480078401C1949087008460078B1
:10058000052804DA0821154800F022FA21E0144871
:100590000078092807DB00201149087008210F485E
:1005A00000F014FA15E00E480078052811DD082146
:1005B0000A4800F00BFA0CE00648007A022804D141
:1005C0000821064800F004FA03E00821034800F07F
:1005D000FDF910BDF80600205C0000200004004872
:1005E0005D00002010B50120800300F0D7F800283E
:1005F00003D00120800300F0CBF810BD10B55748A0
:10060000807D002804D18021554800F0DFF92EE0DC
:100610005248807D012804D18021514800F0D8F94A
:1006200025E04E48807D022821D14E480078401CAC
:100630004C49087008460078052804DA80214848AB
:1006400000F0C6F913E047480078092807DB0020CE
:10065000444908708021424800F0B8F907E0414859
:100660000078052803DD80213D4800F0AFF93B48C4
:1006700016304078002804D14021394800F0A6F90E
:1006800030E0364816304078012804D14021344803
:1006900000F09EF926E0314816304078022821D13A
:1006A00030484078401C2F4948700846407805285B
:1006B00004DA40212A4800F08BF913E029484078F9
:1006C000092807DB0020274948704021244800F012
:1006D0007DF907E023484078052803DD40212048C4
:1006E00000F074F91D4816308078002804D12021CC
:1006F0001B4800F06BF930E018481630807801286C
:1007000004D12021164800F063F926E01348163082
:100710008078022821D113488078401C11498870C4
:1007200008468078052804DA20210D4800F050F9A9
:1007300013E00C488078092807DB002009498870FD
:100740002021074800F042F907E006488078052894
:1007500003DD2021024800F039F910BDD806002041
:10076000000400485800002010B5012000F016F8E1
:10077000002802D0012000F00BF8022000F00EF853
:10078000002802D0022000F003F810BD70470000DE
:100790000149486170470000000401400146002003
:1007A000044A52690A40002A01D0012000E00020DA
:1007B0007047000000040140002120498279002A8E
:1007C00035D00A46126803689A430B461A600A46F7
:1007D000526803689A430B465A60027951180A68B6
:1007E00003681A430A60154A926803689A43134BD8
:1007F0009A601A46D26803689A43104BDA604279CD
:10080000102A0CD11A46926803681A430B4B9A605F
:100810001A46D26803681A43084BDA600DE00749AC
:10082000427951180A6803681A430A6005E00279A0
:1008300051180A6803689A430A607047000401402F
:1008400000B585B00121480400F0F8FE01218805BB
:1008500000F0F4FE0121084600F010FF01208002A4
:100860000090012168460171002181710121C1714F
:1008700069460920C00600F035F8012189020920E7
:10088000C00600F0A5F80120009000216846017123
:1008900001218171032141710121C17169460F4814
:1008A00000F020F80021052001F01EF8012003903F
:1008B0000021684601740C2141740121817403A850
:1008C000FFF77AFF0521684601720021417201217C
:1008D000817202A800F0EEFC05B000BD00140048D3
:1008E00070477047F0B50A4600210023002400BF7E
:1008F0003DE001258D402B4615681D402C469C424D
:1009000034D11579012D02D01579022D16D18568C3
:100910004F000326BE40B543856055794E00B54073
:10092000866835438560858801268E40B54385807D
:10093000858896798E40B6B23543858005684F002C
:100940000326BE40B543056015794E00B5400668E4
:1009500035430560C5684F000326BE40B543C560FA
:10096000D5794E00B540C6683543C560491C10298D
:10097000BFD3F0BDF0B5002300244D07EE0E1546A1
:10098000B5402B46CD10AE0005462035AD594E077B
:10099000F70E0F26BE40B543CE10B60007462037EF
:1009A000BD51CD10AE003D46AD591D432C46CD1076
:1009B000AD003E467451F0BD02460020138A0B4044
:1009C000002B01D0012000E0002070470185704716
:1009D000816170471CB501210720400400F02EFE04
:1009E0000121880500F02AFE0121084600F046FE9C
:1009F000012000900121684601710321417100210D
:100A000081710121C17169460920C006FFF76AFFA3
:100A100010200090012168460171032141710021DD
:100A200081710121C17169460920C006FFF75AFF93
:100A300010210920C006FFF7C9FF202000900021E7
:100A40006846017101218171032141710121C17148
:100A500069460920C006FFF745FF0022062109204C
:100A6000C006FFF787FF4020009002216846017111
:100A7000032141710021817169460920C006FFF7F9
:100A800031FF40200090012168460171032141712E
:100A9000002181710121C17169460920C006FFF75B
:100AA00021FF40210920C006FFF792FF802000901F
:100AB00000216846017101218171032141710121E9
:100AC000C17169460920C006FFF70CFFFF20013005
:100AD000009000216846017101218171032141715B
:100AE0000121C17169460920C006FFF7FBFE012004
:100AF000009000216846017101218171032141713B
:100B00000121C17169466648FFF7ECFE02200090A2
:100B10000021684601710121817103214171012188
:100B2000C17169465E48FFF7DDFE0120400200907A
:100B30000021684601710121817103214171012168
:100B4000C17169460920C006FFF7CCFE0120800272
:100B500000900021684601710121817103214171DA
:100B60000121C17169460920C006FFF7BBFE0120C3
:100B7000C0020090002168460171012181710321AA
:100B800041710121C17169460920C006FFF7AAFE23
:100B9000012000030090002168460171012181714C
:100BA000032141710121C17169460920C006FFF787
:100BB00099FE0120C00300900121684601710321C4
:100BC0004171002181710121C17169460920C0066E
:100BD000FFF788FE0121C9030920C006FFF7F6FED2
:100BE0000820009001216846017103214171002114
:100BF00081710121C17169462948FFF773FE0821FF
:100C00002748FFF7E3FE102000900121684601719C
:100C100003214171002181710121C1716946204880
:100C2000FFF760FE10211E48FFF7D0FE2020009045
:100C30000121684601710321417100218171012167
:100C4000C17169461648FFF74DFE20211448FFF791
:100C5000BDFE4020009001216846017103214171D1
:100C6000002181710121C17169460D48FFF73AFEEB
:100C700040210B48FFF7AAFE802000900121684622
:100C8000017103214171002181710121C171694606
:100C90000348FFF727FE80210148FFF797FE1CBDA0
:100CA0000004004800BFFEE70246002100202A4B56
:100CB0001B78302B08DB284B1B78392B04DC264BA8
:100CC0001B78303B99B203E0234B1B78373B99B23A
:100CD0000B07180C204B5B78302B08DB1E4B5B7826
:100CE000392B04DC1C4B5B78303B99B203E01A4B88
:100CF0005B78373B99B20B06190C03460B43184639
:100D0000154B9B78302B08DB134B9B78392B04DC7D
:100D1000114B9B78303B99B203E00F4B9B78373BEC
:100D200099B20B05190C03460B4318460A4BDB78A6
:100D3000302B08DB084BDB78392B04DC064BDB78E7
:100D4000303B99B203E0044BDB78373B99B2034662
:100D50000B43184670470000003300080148024961
:100D600008607047CCCC00000030004001480249C8
:100D700008607047AAAA000000300040014948609E
:100D80007047000000300040014988607047000053
:100D9000003000400149086070470000003000400A
:100DA00010B528480078401C26490870264800786D
:100DB000401C2549087025480088401C23490880AC
:100DC00023480088401C22490880FF210131092066
:100DD000C006FFF7F1FD002807D11B4800780F2857
:100DE0000DDB00201849087009E000201749088031
:100DF0001549087017480088401C16490880134898
:100E000000884B21090188420ADD1348407C0028F4
:100E100006D000200D490880104A012100F0DCFABC
:100E20000C4800880E4988420BD10B48407C0028B2
:100E300007D0002007490880084A521E012100F00F
:100E4000CBFA10BD26000020270000202A00002039
:100E5000280000202C000020F806002004070000D5
:100E60003075000010B52A480078401C28490870E9
:100E700028480078401C2749087027480088401CF3
:100E80002549088025480088401C24490880012104
:100E90002348FFF791FD002812D11E4800780A2848
:100EA00005DB00201B49087001211E48C17300208A
:100EB000194908801C480088401C1B49088005E02F
:100EC00000201449087000211648C1731248008898
:100ED000164988420ADD1348407C002806D00020CD
:100EE0000D490880124A012100F076FA0E48008868
:100EF000104988420BD10B48407C002807D00020C5
:100F0000094908800A4A521E012100F065FA10BD05
:100F10001D0000201E0000202200002020000020D4
:100F200000040048F806002024000020E02E000005
:100F300004060000307500001CB50024002000905D
:100F40000190012189020920C006FFF735FD002824
:100F500001D1012100E00021684601708848C17B71
:100F60006846417080210920C006FFF725FD002852
:100F700001D1012000E000206946887001210903A9
:100F80000920C006FFF718FD002801D1012000E06C
:100F900000206946C8700121C9020920C006FFF778
:100FA0000BFD002801D1012000E0002069460871F6
:100FB00002217448FFF700FD002801D1012000E064
:100FC000002069464871012149020920C006FFF747
:100FD000F3FC002801D1012100E000216846817165
:100FE00020210920C006FFF7E7FC01466846C171D1
:100FF0004079002824D068464078002820D06248F4
:101000000078401C6049087008460078032809DD14
:101010005E480078002805D101205C490870002056
:101020005949087059480078012808D102205749C9
:1010300008700D2212020121002000F0CDF91CBD24
:1010400000205149087051480078022808D1504AC0
:101050000121002000F0C0F900204C490870EEE7A3
:1010600000204A490870002484E06846005D00289A
:1010700031D143482038C07F0121A14088434049F5
:101080002039C8770020434908554348005D401C7B
:101090004149085501204149087000206100404A3B
:1010A00050523D48005D032862DD00203A49085552
:1010B0003C48005D6946095D884259D0601D0002C8
:1010C000401C82B20121002000F086F96846005DD4
:1010D000344908554CE02A482038C07F0121A140FE
:1010E0000843C1B226482038C1772A48005D401C19
:1010F0002849085500202849085560002849085A01
:10110000401C6100264A50522248005D03282FDD12
:1011100000202049085560001146085A322816DD83
:101120000020610050521D480078022820D0022083
:101130001A490870012C1BD0022C19D0601D000226
:10114000801C82B20121002000F046F910E0154811
:10115000005D6946095D88420AD0601D0006020CE8
:101160000121002000F038F96846005D0D4908555E
:10117000601CC4B2082C00DA77E700BF5FE700000C
:10118000F806002000040048460000204700002028
:10119000010D0000360000203E0000204800002025
:1011A0008C0000201400002010B532480078002880
:1011B00000D010BD01202F49087081020920C0060F
:1011C000FFF7FAFB002801D1012000E000202A49A6
:1011D00008702A48C07B487080210920C006FFF7AC
:1011E000EBFB002801D1012000E00020224988709B
:1011F000012109030920C006FFF7DEFB002801D109
:10120000012000E000201C49C8700121C90209200A
:10121000C006FFF7D1FB002801D1012000E000202B
:101220001549087102211648FFF7C6FB002801D1B5
:10123000012000E0002010494871012149020920E5
:10124000C006FFF7B9FB002801D1012000E0002013
:101250000949887120210920C006FFF7ADFB064926
:10126000C871002105482038C1772030017000BFC7
:101270009FE700001C00002014000020F80600205A
:101280000004004810B50449887C00F0B9FBFFF762
:10129000B5F9FFF735F910BDD806002030B5044682
:1012A000002303E02170641C5D1CABB29342F9DBA8
:1012B00030BD704700218278002A27D0184A0323C6
:1012C0001B02D21803789B109B00D158027892071A
:1012D000D30EFF229A400B46934319464278920759
:1012E000120E03789B07DB0E9A4011430C4A03232E
:1012F0001B02D21803789B109B00D1500278D306B2
:10130000DB0E01229A40064B1A6007E00278D306F2
:10131000DB0E01229A40024B80331A6070470000B6
:1013200000E100E0002252214143044B5A54802244
:1013300052214143C9184A70704700009C000020A8
:1013400070B5014600201C4D2870522048431B4DAB
:10135000285C43065B0E5220484340194078420601
:10136000520E5220484340194078802528400446B8
:10137000002C13D152204843104D4019801C950079
:1013800040190D4D06882E8040886880501CC2B2DE
:10139000142A00DB0022934200D10124002C01D04A
:1013A0008020024352204843044D2B54522048438E
:1013B00040194270004870BD4A0000209C00002087
:1013C00010B5002404E02046FFF7ACFF601CC4B257
:1013D000072CF8DB10BD0000F8B50B466E463370E5
:1013E0007280522646431A4FBE5D7106490E522640
:1013F0004643BE5D80273E40354652264643144F45
:10140000F61976787406640E002D13D152264643E1
:10141000F619B61C8F00F7196E4636883E806E4668
:1014200076887E804E1CF1B2142900DB0021A14297
:1014300000D10125002D01D080263143522646439C
:10144000034FB95552264643F6197470F8BD000093
:101450009C00002010B502460020154B186880083B
:101460008000034613431846114B1860114B1B694B
:10147000042423430F4C2361012907D130BF2346A5
:101480001B690424A3430B4C23610FE0022907D1FD
:1014900020BF084B1B690424A343064C236105E0CD
:1014A000044B1B6902242343024C236110BD00003E
:1014B0000070004000ED00E07047000010B54748A4
:1014C0000078030000F0C4FD09060E1D2A323B47D8
:1014D0004855870041480078401C4049087000206A
:1014E000488079E03D4840887D21C900884200DC81
:1014F00072E000203949488008460078401C087096
:101500006AE0364840887D210901884200DC63E0BA
:1015100032480078401C314908705DE000202F49B6
:10152000488008460078401C087055E000202B4990
:10153000C880488008460078401C08704CE0274866
:1015400040882749884200DC46E024480078401C57
:101550002249087040E03FE0204840887D21C900D2
:10156000884200DC38E000201C49488008200870D0
:1015700032E01A484088642800DA2DE0FFF760F96D
:1015800000F0C4FA00F0D2FA0120164948707D211B
:10159000C90015480068FEF743FE0446601E134963
:1015A000884201D901200CE0601E114948610321E5
:1015B000081F00F05BFD00200D49886107200861CD
:1015C0000020002801D000BFFEE705200349087075
:1015D0000020488000E000BF00BF10BDDC020020FA
:1015E00088130000B806002000000020FFFFFF0065
:1015F00000E000E00A4840880A49884204D00848D0
:101600004088401C064948800548C08805498842F2
:1016100004D00348C088401C0149C88070470000BE
:10162000DC020020FFFF0000002003490870488012
:1016300008718860C8807047DC020020002905D04E
:10164000054A52690243044B5A6104E0024A526956
:101650008243014B5A61704700100240002905D0B7
:10166000054AD2690243044BDA6104E0024AD269B6
:101670008243014BDA61704700100240002905D017
:10168000054A92690243044B9A6104E0024A926956
:101690008243014B9A61704700100240FEB5044638
:1016A0000025002600200290019000900027864827
:1016B00040680C2108400546002D06D0042D07D0B7
:1016C000082D08D00C2D2CD128E0804820602BE07C
:1016D0007E48206028E07C4840680F21890408404B
:1016E0000646794840680321C90308400290B00CBF
:1016F000861C0298002803D17548374647430BE003
:101700007148C06A0007000F401C01906F480199A2
:10171000FEF786FD70430746276005E06D482060B0
:1017200002E06A48206000BF00BF67484068F021BF
:10173000084005462D096848405D009020680099E2
:10174000C8406060604840680721090208400546BB
:101750002D0A6148405D009061680098C140A16019
:101760005948006BFF2101310840884202D05B4894
:10177000E0600DE054484068012189030840884238
:1017800003D0A0684008E06002E0A0688008E06044
:101790004D48006B40210840402802D0504820614D
:1017A00002E00120C00320614748006B102108407F
:1017B000102802D04548606101E02068606142481D
:1017C000006B8007800F002802D1A068A06119E09B
:1017D0003D48006B8007800F012802D12068A0617E
:1017E00010E03948006B8007800F022802D1800387
:1017F000A06107E03448006B8007800F032801D107
:101800003248A0613048006B0321090408400028D9
:1018100002D1A068E06120E02B48006B032109049D
:10182000084001210904884202D12068E06114E0E7
:101830002548006B0321090408400121490488421E
:1018400002D18010E06108E01F48006B0321090409
:101850000840884201D11D48E0611B48006B03210C
:1018600089040840002802D1A068206220E01648C0
:10187000006B03218904084001218904884202D1B8
:101880002068206214E01048006B0321890408409E
:101890000121C904884202D10011206208E00A48EF
:1018A000006B032189040840884201D10748206267
:1018B0000548006B80210840802802D005486062FE
:1018C00000E06762FEBD00000010024000127A00D6
:1018D00000093D00006CDC027B000020809FD500E9
:1018E000128000007047000030B500228B071C0FEB
:1018F0000F23A3401A460B4B8C10A4001B59934393
:10190000084C8D10AD00635123468C10A4001B5968
:101910008C07250F0446AC402343024C8D10AD00CC
:10192000635130BD080001400CB5002001900090CB
:10193000304800680121090408432E49086000BFAF
:101940002C48006801214904084000900198401C7F
:1019500001900098002803D1274901988842EFD1CF
:1019600024480068012149040840002802D00120D1
:10197000009001E0002000900098012839D111204A
:101980001E4908601B4840681A494860084640687C
:101990004860084640687F21C9038843154948606C
:1019A0000846406811210904084312494860084666
:1019B00000680121090608430E49086000BF0D4870
:1019C00000680121490608400028F8D0094840680D
:1019D00080088000074948600846406802210843A3
:1019E0000449486000BF034840680C2108400828AB
:1019F000F9D10CBD00100240FFFF000000200240A2
:101A000010B50446002C05D140210920C006FEF780
:101A1000DDFF2EE0012C05D140210920C006FEF794
:101A2000D7FF26E0022C24D112480078401C11492F
:101A3000087008460078052805DA40210920C0060C
:101A4000FEF7C6FF15E00B480078092808DB4021A7
:101A50000920C006FEF7BAFF00200649087008E01A
:101A600004480078052804DD40210920C006FEF75F
:101A7000ADFF10BD5700002010B51C480078FF28AE
:101A800004D01A480078401C18490870184800789B
:101A9000FF2804D016480078401C154908701548E6
:101AA0000078FF2804D013480078401C11490870C2
:101AB00011480078FF2804D00F480078401C0E49D8
:101AC00008700E48807BFF2805D00C48807B401CA6
:101AD000C1B20A488173FFF78DFDFEF7ADFC0848DF
:101AE0000078401C0649087010BD0000520000201C
:101AF000530000205400002055000020F80600206C
:101B00005600002010B5FFF7B7FF10BD10B500203C
:101B100005490861886101210807FFF79FFD012140
:101B20000846FFF797FC10BD00E000E010B51B4829
:101B300000680121084319490860084640681849AF
:101B4000084016494860084600681649084013498D
:101B50000860084600680121890488430F4908602D
:101B6000084640683F21090488430C4948600846FC
:101B7000C06A00090001C8620846006BFF215431A9
:101B80008843064908630846406B400840004863A4
:101B900000208860FFF7C8FE10BD00000010024062
:101BA0000CB8FFF8FFFFF6FE10B500F047F910BDC6
:101BB00001627047002904D0026801231A430260C1
:101BC00003E002685208520002607047024600209B
:101BD000D3690B40002B01D0012000E000207047AA
:101BE000F8B503460024002600960025002018467C
:101BF0000E04340ECEB200960127009EB7403D463B
:101C0000022C01D1001D02E0032C00D10830002A73
:101C100003D006682E43066002E00668AE43066005
:101C2000F8BD0000F0B58BB004460D46002700203B
:101C30000A90002620684008400020606668032162
:101C40000903304688430646A8680643666026684E
:101C50002D480640E9686868084329690843064337
:101C60002660A66803210902304688430646686953
:101C70000643A6606846FFF711FD2448844202D15E
:101C800006980A900DE02248844202D107980A90F3
:101C900007E02048844202D108980A9001E00298A7
:101CA0000A9020680121C903084000280CD0296847
:101CB0000A9A5000FEF7B4FA074629680A9A5000BB
:101CC000FEF7AEFA0E4609E029680A98FEF7A8FA70
:101CD000074629680A98FEF7A3FA0E4628684008C6
:101CE000B04200D87F1C20680121C90308400028A9
:101CF00006D03807460F38460749084030430746A4
:101D0000A7810BB0F0BD0000F3E9FFFF00380140F0
:101D10000044004000480040F0FF00000146888C6D
:101D2000C005C00D7047CA05D20D0285704700007E
:101D300000B589B0182101A8FEF770FA00F010FB79
:101D400001214804FFF77AFC01218803FFF796FC84
:101D5000012202210920C006FEF70CFE0122032108
:101D60000920C006FEF706FE0C200790022108A8F5
:101D700001700321417001218170C17007A9092000
:101D8000C006FEF7AFFDE120400201900020029066
:101D90000390049006900C20059001A90B48FFF7D2
:101DA00041FF01210948FFF705FF012208490748C3
:101DB000FFF716FF012207490448FFF711FF4021F2
:101DC0000248FFF7F5FE09B000BD000000380140F1
:101DD0000501050006010600F7B50546164C00F0A2
:101DE000B3FA002824D160784101201D465C1E2EE4
:101DF00000DD1E262E706D1C701CC6B2002709E087
:101E000060784101201D0918781C085C28706D1C41
:101E1000781CC7B2B742F3DB6078401C6070607812
:101E2000142801DB0020607000210298017002E09C
:101E3000022102980170FEBDEC02002070B5002561
:101E4000464C40214648FFF7C1FE002839D0052006
:101E5000C00120180079002827DD0520C0012018C6
:101E60000079401E0521C901611808710520C001D3
:101E700020188079FA2804DB00200521C9016118A7
:101E800088710520C001201882790520C001201822
:101E90008079401C0523DB01E31898713148201834
:101EA000815C2F48FFF73FFF07E00520C0012018A5
:101EB00040790521C9016118887140212848FFF740
:101EC00077FE20212648FFF781FE002844D02448D1
:101ED000FFF724FFC5B224480078002802D001286B
:101EE00031D107E0242D02D101201F4908700120C3
:101EF000E0702CE0232D17D1232120784201201DF2
:101F00001018E2788154E17820784201201D815434
:101F10002078401C20702078142801DB00202070DD
:101F20000020114908700DE0242D02D10120E0703D
:101F300008E020784101201D0818E1784554E07838
:101F4000401CE07003E000200749087000BF00BF9C
:101F500020210348FFF72CFE70BD0000EC0200209A
:101F6000003801408702000062000020F8B50546F5
:101F70000E46344C002E01D10420F8BD00F0E4F9E7
:101F8000074625E00520C00120180079401C0521E6
:101F9000C901611808710520C00120184079FA288C
:101FA00004DB00200521C90161184871287805214A
:101FB000C901611849790522D201A2185279521C2F
:101FC0000523DB01E3185A711F4AA21850546D1CF7
:101FD0003046711ECEB20028D4D1002F30D005205B
:101FE000C00120180079002808D00520C001201861
:101FF0000079401E0521C901611808710520C00142
:1020000020188079FA2804DB00200521C901611815
:1020100088710520C001201880790522D201A218FC
:102020009279521C0523DB01E3189A71064AA21823
:10203000115C0648FFF777FE08210448FFF7B8FD5A
:1020400000209AE7EC0200208702000000380140DF
:1020500030B47446641E2578641CAB4204D3635DBF
:102060005B00E31830BC18471D46F8E710B50028A0
:1020700019DB1A4A03231B02D21883089B00D2588B
:102080008307DC0EFF23A3409A438B071B0E8407B4
:10209000E40EA3401A43114B032424021B198408A5
:1020A000A4001A5118E00E4A03071B0F083B9B08B7
:1020B0009B00D2588307DC0EFF23A3409A438B0773
:1020C0001B0E8407E40EA3401A43054B0407240F9C
:1020D000083CA408A4001A5110BD000000E100E073
:1020E0001CED00E010B5002819DB1A4A03231B027F
:1020F000D21883089B00D2588307DC0EFF23A3402D
:102100009A438B071B0E8407E40EA3401A43114B1E
:10211000032424021B198408A4001A5118E00E4A53
:1021200003071B0F083B9B089B00D2588307DC0E5C
:10213000FF23A3409A438B071B0E8407E40EA340A2
:102140001A43054B0407240F083CA408A4001A51A5
:1021500010BD000000E100E01CED00E000F0B0F870
:1021600000F094F800F082F800F0D0F800F06CF87D
:1021700032E0FEF7FBFD19480078052809DB002056
:1021800016490870FEF768F9FEF76CFEFEF708FEC8
:1021900022E013480078232807DB0020104908704C
:1021A000FEF722F9FEF7C8FE16E00E480078642814
:1021B00009DB00200B490870FFF780F9FEF790FB60
:1021C000FFF760F808E008480078232803DB0020C8
:1021D0000549087000E000BFCBE700005200002076
:1021E0005300002054000020550000200021044826
:1021F0000178405C232801D1012070470020FCE7D2
:102200007006002070B5054600240026E9000C4A3F
:102210005058FDF7C3FFC6B200BF0CE0E800084904
:102220000858015D601C074A105C814201D0002003
:1022300070BD601CC4B2B442F0DB0120F8E70000BE
:10224000982900087006002010B50748FEF7A2FD87
:102250000520FEF793FD7D20C000FEF795FDFEF7FB
:1022600085FDFEF77BFD10BD5555000000B58BB018
:1022700001A8FFF713FA0121684641701B21017084
:1022800001218170FFF716F80BB000BD10B50024D6
:10229000FEF7A0FBFFF74CFD06480468002C07D0B2
:1022A0000548844204D02046FEF7FEFC034988819D
:1022B00010BD000000330008FFFFFF00F8060020FB
:1022C00010B57D21C9000E480068FDF7A9FF04463E
:1022D000601E0C49884201D901200CE0601E0A49A9
:1022E00048610321081FFFF7FDFE002006498861B1
:1022F000072008610020002801D000BFFEE710BDC4
:1023000000000020FFFFFF0000E000E010B500200B
:102310000949087009490870094908700949087095
:10232000FFF782F9FEF740FFFEF7C8F8FEF7D9FA8B
:10233000FFF746F810BD00005200002053000020B7
:1023400054000020550000200448007803494978D3
:10235000884201D1012070470020FCE7EC020020F8
:1023600003480021017041708170C1707047000006
:10237000EC02002010B50A484079492805D1002216
:1023800002211046FFF728F808E005484079562852
:1023900004D1002203211046FFF71EF810BD0000F3
:1023A000700600200648407A3038C1B20548C17135
:1023B0000348807A3038C1B2024801727047000089
:1023C00070060020F80600200A48407A3038C1B272
:1023D000094881750748807A3038C1B206481630FE
:1023E00041700448C07A3038C1B203481630817059
:1023F0007047000070060020D8060020704710B516
:10240000002202211046FEF7E7FF10BD70470000D2
:1024100010B50A48807A302805D110210920C0065D
:10242000FEF7D4FA08E00548807A312804D110215B
:102430000920C006FEF7CCFA10BD0000700600208F
:1024400010B58D48407930380300FFF701FE0504D0
:102450003A70A6DC39008849C97930390A225143DB
:10246000854A127A303A891808026421FDF7E2FEA3
:10247000C1B28248C1728049497A30390A22514337
:102480007D4A927A303A891808026421FDF7D2FE1B
:10249000C1B27A4801737849C97A30390A22514366
:1024A000754A127B303A891808026421FDF7C2FE92
:1024B000C1B272488172007C012108436F490874DF
:1024C000D7E06D49C97930390A2251436A4A127AF4
:1024D000303A891808026421FDF7ACFEC1B26748A2
:1024E00081736549497A30390A225143624A927AA6
:1024F000303A891808026421FDF79CFEC1B25F489A
:10250000C1735D49C97A30390A2251435A4A127B54
:10251000303A891808026421FDF78CFEC1B2574891
:102520004173007C0221084354490874A1E05249D8
:10253000C97930390A2251434F4A127A303A891800
:1025400008026421FDF776FEC1B24C4881704A4909
:10255000497A30390A225143474A927A303A8918E7
:1025600008026421FDF766FEC1B24448C1704249C9
:10257000C97A30390A2251433F4A127B303A8918CE
:1025800008026421FDF756FEC1B23C484170007C50
:1025900004210843394908746BE03749C979303957
:1025A0000A225143344A127A303A891808026421C7
:1025B000FDF740FEC1B2314841712F49497A3039A7
:1025C0000A2251432C4A927A303A8918080264212F
:1025D000FDF730FEC1B2294881712749C97A3039E7
:1025E0000A225143244A127B303A89180802642196
:1025F000FDF720FEC1B221480171007C082108438B
:102600001E49087435E01C49C97930390A22514302
:10261000194A127A303A891808026421FDF70AFE35
:10262000C1B2164801721449497A30390A2251431D
:10263000114A927A303A891808026421FDF7FAFDAE
:10264000C1B20E4841720C49C97A30390A2251434D
:10265000094A127B303A891808026421FDF7EAFD25
:10266000C1B20648C171007C1021084303490874B7
:1026700000BF00BF10BD000070060020D80600207B
:102680000D48007A2C2816D10B48807A462812D1A2
:102690000948C07A23280ED10748407A312803D14F
:1026A00001210648417406E00348407A302802D1EF
:1026B000002102484174704770060020F80600208F
:1026C00010B50024164880793038C4B2002C18D1D7
:1026D0001348017A1348C174C07C302806D1012107
:1026E000C9030920C006FEF771F917E00D48C07C48
:1026F000312813D10121C9030920C006FEF768F96A
:102700000CE0012C05D10648017A064813304170CF
:1027100004E00348017A03481330817010BD0000C3
:1027200070060020D80600200B484079302803D1DD
:1027300000210A4841740EE007484079312803D14E
:1027400001210648417406E003484079322802D14D
:10275000022102484174704770060020D80600200C
:10276000002002490870024948707047DC020020CE
:10277000B8060020002002490870024948707047DE
:10278000DC020020B8060020002005498979303994
:10279000C8B2022800DD0220024988747047000098
:1027A00070060020D806002010B500220421104633
:1027B000FEF712FE10BD000070B50646002400258D
:1027C0000E4C24202070641C49202070641C44207E
:1027D0002070641C2C202070641C00BF01E0681C69
:1027E000C5B20F2DFBDB31202070641C232020702C
:1027F000641C15210148FFF7B9FB70BD8E0600204F
:1028000070B505460024324C24202070641C4B20F7
:102810002070641C45202070641C59202070641CAA
:102820002812082803D13B202070641C2DE02812B8
:10283000092803D13C202070641C26E028120A28B5
:1028400003D13D202070641C1FE028120B2803D107
:102850003E202070641C18E028120D2803D13F2070
:102860002070641C11E028120C2803D14020207035
:10287000641C0AE028120E2803D138202070641C42
:1028800003E0281230302070641C2C202070641C5F
:102890000121104841722812052807DAE8B20228FF
:1028A00004D1FF20000205400120054328463030B6
:1028B0002070641C23202070641C00202070641C85
:1028C00009210348FFF752FB00210248817370BDC4
:1028D0008E060020F806002000BF704770B506463F
:1028E000002400250F4C24202070641C56202070EA
:1028F000641C2C202070641C00BF05E00A48405D69
:102900002070641C681CC5B20F2DF7DB46202070B8
:10291000641C23202070641C14210248FFF726FB4E
:1029200070BD00008E0600208029000870B50646A4
:1029300000240025104C24202070641C5620207098
:10294000641C2C202070641C00BF05E00B48405D17
:102950002070641C681CC5B20F2DF7DB4620207068
:10296000641C23202070641C002020701421024865
:10297000FFF7FCFA70BD00008E06002080290008D9
:10298000535A443130313031323530323039310000
:102990002448454152540000982A0008FD230008AD
:1029A000802A000861270008542A000875270008BB
:1029B0002C2A00080D240008382A000841240008A9
:1029C000482A000889270008A02A0008C126000814
:1029D0007C2A000829270008502A0008FF23000845
:1029E000402A0008C9230008302A0008A52300084F
:1029F000682A0008752300088C2A000811240008A2
:102A00006C2A0008FD230008602A000881260008BF
:102A1000742A0008A9270008D928000801280008FE
:102A2000B9270008DD2800082D2900084D4943007A
:102A300043414C4C4C4544004E4C45440000000082
:102A4000444F4F524C454400554C45440000000053
:102A50004944000053595355504441544500000027
:102A60004F4C434845434B0041534B0043414C4C72
:102A70000000000056455253494F4E005349500044
:102A80005359535245534554000000004E4554528B
:102A90004553455400000000484541525400000091
:102AA00052454C4159000000083300080000002046
:102AB0008C00000004010008943300088C00002002
:102AC000E40C0000200100080000000000000000ED
:102AD00000000000000000000000000000000000F6
:102AE00000000000000000000000000000000000E6
:102AF00000000000000000000000000000000000D6
:102B000000000000000000000000000000000000C5
:103300004633303100000000006CDC020000000099
:103310000000000001020304060708090000000085
:10332000000000000000000000000000000000009D
:10333000000000000000000000000000000000008D
:10334000000000000000000000000000000000007D
:10335000000000000000000000000000000000006D
:103360000000000000000000000000000000C0A8F5
:1033700001D3C0A801010000C0A801AA00000000FC
:103380000000000000000001020304010203040623
:043390000708090021
:04000005080000C12E
:00000001FF
